S011000048656E64694374726C2E7372656396
S11300000C9434000C9451000C9451000C94510045
S11300100C9451000C9451000C9451000C94510018
S11300200C9451000C9451000C9451000C94510008
S11300300C9451000C94A1060C9451000C945100A2
S11300400C9451000C9451000C945A070C945007D2
S11300500C9446070C9482000C9451000C945100AB
S11300600C9451000C94510011241FBECFEFD8E022
S1130070DEBFCDBF12E0A0E0B1E0E2E0FCE102C0EF
S113008005900D92A832B107D9F722E0A8E2B2E0B8
S113009001C01D92AD3AB207E1F70E94D1020C945F
S11300A0FF0D0C940000909339028093380228E1EC
S11300B031E041E050E060E170E08AE292E00E94C9
S11300C01E01E4E6F0E080818E7F8083EAE7F0E0C1
S11300D08081876880830895ECE7F0E09081907FC9
S11300E090648F70982B9083EAE7F0E09081986495
S11300F0908380933A0281E090E090932902809368
S1130100280208951F920F920FB60F9211242F9375
S11301103F934F935F936F937F938F939F93AF938B
S1130120BF93EF93FF93CF93DF93CDB7DEB72597BC
S1130130DEBFCDBF10922902109228028091780070
S11301402091790090917A00906190937A0092E0E6
S1130150998390913A029A8390E0922B9C838B83AB
S1130160BE016F5F7F4F80913802909139020E94E7
S113017063018AE292E00E94F201892B51F4BE01EC
S11301806B5F7F4F8AE292E00E94AC018D810E94F6
S11301906C000F900F900F900F900F90DF91CF9104
S11301A0FF91EF91BF91AF919F918F917F916F914B
S11301B05F914F913F912F910F900FBE0F901F9021
S11301C01895CF93DF931F92CDB7DEB789838091C3
S11301D0280290912902892B21F489810E946C00C4
S11301E007C0BE016F5F7F4F8AE292E00E94630105
S11301F00F90DF91CF910895F89480913B029091F4
S11302003C02019690933C0280933B0208958091B6
S11302103B0290913C02892B81F080913B029091AA
S11302203C02019790933C0280933B0280913B02F5
S113023090913C02892B09F4789408958F929F92AF
S1130240AF92BF92CF92DF92EF92FF920F931F93E0
S1130250CF93DF93EC017B014A015901198618867B
S11302601B861A861F821E827B836A835D834C836E
S1130270CB01880F991F0E94A6089983888300E008
S113028010E00E151F0581F0C801880F991FC88062
S1130290D980C80ED91EC4010E94A608F601918314
S11302A080830F5F1F4FEDCFBD86AC86DF91CF916A
S11302B01F910F91FF90EF90DF90CF90BF90AF9080
S11302C09F908F9008950F931F93CF93DF93EC012A
S11302D08B010E94FC002E813F818A819B8128171B
S11302E0390768F5D8019D01201B310B8C819D8154
S11302F02817390780F4E885F9854D91EE0FFF1F23
S113030088819981E80FF91F80819181FC01E20FB6
S1130310F31F4083E8CF888599850196998788875C
S11303208E819F8101969F838E83288539858A815A
S11303309B812817390731F41986188603C0C0E059
S1130340D0E002C0C1E0D0E00E940701CE01DF91FD
S1130350CF911F910F9108950F931F93CF93DF9324
S1130360EC018B010E94FC008E819F81892B69F135
S1130370D801CD01801B910B2C813D8182179307FD
S113038080F4EA85FB85EE0FFF1F28813981E20F97
S1130390F31F20813181F901E80FF91F80818D93CA
S11303A0E8CF8A859B8501969B878A878E819F816A
S11303B001979F838E832A853B858A819B81281799
S11303C0390731F41B861A8603C0C0E0D0E002C0AE
S11303D0C1E0D0E00E940701CE01DF91CF911F91CF
S11303E00F910895CF93DF93EC010E94FC000E80DF
S11303F0DF81C02D0E94070181E090E0CD2B11F038
S113040080E090E0DF91CF9108958FEF8093B80062
S11304101092B900089594EA9093BC009091BC00A6
S113042097FFFCCF9091B900987F983019F081E242
S113043091E017C0880F682B6093BB0084E8809319
S1130440BC008091BC0087FFFCCF8091B900887FFD
S1130450883129F4FA01240F351F94E805C081E39B
S113046091E00E94400B14C0E217F30789F08191D8
S11304708093BB009093BC008091BC0087FFFCCFAD
S11304808091B900887F883279F383E491E0E9CFE1
S113049084E98093BC0008950F931F93CF93DF9357
S11304A000D000D0CDB7DEB78C0190934202809388
S11304B041028091140190911501A0911601B0910F
S11304C0170189839A83AB83BC83809149029091FD
S11304D04A02892BE9F0E1E0F0E00115110511F47D
S11304E0E0E0F0E0EE0FFF1F81E090E08C0F9D1F35
S11304F0E80FF91F81818F9380818F9386E591E0C6
S11305009F938F930E942A0B0F900F900F900F9040
S113051061E070E0012B11F460E070E087E090E0AE
S11305200F900F900F900F90DF91CF911F910F912B
S11305300C9482060F931F93CF93DF9300D0CDB713
S1130540DEB78C0180933D0210933E0280914902F4
S113055090914A02892B61F01F930F938FE691E0EB
S11305609F938F930E942A0B0F900F900F900F90E0
S113057019821A8242E050E0BE016F5F7F4FC801CA
S11305800E9466069C01AE014F5F5F4F60E080E60B
S11305900E940B020F900F90DF91CF911F910F914A
S11305A00895CF93DF93CDB7DEB76B970FB6F8946A
S11305B0DEBF0FBECDBFF894A8950FB6F894A895EA
S11305C080916000886180936000109260000FBE8B
S11305D02CE131E044E050E068E070E083E992E02F
S11305E00E941E0140E052EC61E070E083E992E079
S11305F00E949E0742E06FEF76EF83E992E00E944B
S1130600160783E992E00E9453000E9405020E94AB
S11306107A0686E091E09093A8028093A7028DEF7A
S113062091E09F938F9382E092E09F938F9387E86A
S113063091E09F938F930E942A0B1D8A1E8A1F8A22
S113064043E050E0BE016B5E7F4F80E090E00E948B
S11306506D069C01AE014B5E5F4F60E080E60E9438
S11306600B026091A7027091A8028DE090E00E94B5
S1130670EE0A6091A7027091A8028AE090E00E94BD
S1130680EE0A6091A7027091A8028AE390E00E94AA
S1130690EE0A60E070E080E00E942E0760E070E007
S11306A082E00E942E0781E090E00E944C02789440
S11306B00F900F900F900F900F900F9010E0812CDF
S11306C0912C58EE452E53E0552E612C712C6FE978
S11306D0C62E61E0D62E7CE9A72E71E0B72E83E901
S11306E092E00E94F201892B09F0EEC2BE016F5E16
S11306F07F4F83E992E00E94AC018989823009F43A
S1130700F7C1833009F424C2813009F0DDC28A893B
S113071020914B0230914C02AE014F5F5F4FFA01C2
S1130720E20FF31F10828D3009F0CDC1598F488F2D
S113073010924C0210924B02012F812F90E0880FEF
S1130740991F9C0129503E4F3B8F2A8F4EE8242E3F
S113075041E0342EE88CF98CF70180818823E1F0A4
S113076090E00E94E60A9C01C7010196998F888F48
S11307702035310509F054C0F70121812F3331F4BC
S1130780F2E0EF0EF11CF98EE88E31C030E0205318
S113079031092A303105F0F060E177E281E00E940E
S11307A02E076091A7027091A8028DE090E00E944C
S11307B0EE0A6091A7027091A8028AE090E00E947C
S11307C0EE0A6091A7027091A8028AE390E00E9469
S11307D0EE0A39C24AE050E0BE01685E7F4F0E94D3
S11307E0C709113009F0B6CFCB010E949A0260917B
S11307F0A7027091A8028DE090E00E94EE0A609139
S1130800A7027091A8028AE090E00E94EE0A80910B
S11308103E028F9380913D028F933F922F924CC161
S11308202335310509F053C0F70121812F3301F538
S1130830F2E0EF0EF11CF98EE88E6091A702709140
S1130840A8028DE090E00E94EE0A6091A7027091E8
S1130850A8028AE090E00E94EE0A809142028F93FF
S1130860809141028F9326E931E03F932F9324C175
S113087030E0205331092A30310508F08DCF4AE0A9
S113088050E0BE01685E7F4F0E94C709113009F035
S113089061CFCB010E944C026091A7027091A80223
S11308A08DE090E00E94EE0A6091A7027091A80288
S11308B08AE090E00E94EE0A809142028F93809138
S11308C041028F93E6E9F1E0FF93EF93F5C02235FF
S11308D0310509F05BC0F701218130E02053310973
S11308E02A30310508F058CF4AE050E0BE01685E76
S11308F07F4F0E94C7096130710511F511112ACF8C
S11309008FEF9FE00E949A0280E090E00E944C02E8
S11309106091A7027091A8028DE090E00E94EE0A17
S11309206091A7027091A8028AE090E00E94EE0A0A
S1130930BF92AF920E942A0B0F900F9001E00ACF52
S1130940672B09F007CF113009F004CF8FEF9FE038
S11309500E949A0280E090E00E944C026091A702FB
S11309607091A8028DE090E00E94EE0A6091A702C7
S11309707091A8028AE090E00E94EE0ABF92AF92C2
S11309800E942A0B0F900F9000E0E4CE243431052E
S113099059F5F701218130E0205331092A3031051E
S11309A008F0FACE4AE050E0BE01685E7F4F0E9434
S11309B0C70970934A02609349026091A70270913B
S11309C0A8028DE090E00E94EE0A6091A702709167
S11309D0A8028AE090E00E94EE0ABF92AF920E94C1
S11309E02A0B0F900F90B6CE29343105E9F4F701A4
S11309F081818F3309F0AECEF2E0EF0EF11CF98E57
S1130A00E88E6091A7027091A8028DE090E00E94A8
S1130A10EE0A6091A7027091A8028AE090E00E9419
S1130A20EE0A22E032E01FC026353105F9F4F70161
S1130A3081818F3309F08ECEF2E0EF0EF11CF98E36
S1130A40E88E6091A7027091A8028DE090E00E9468
S1130A50EE0A6091A7027091A8028AE090E00E94D9
S1130A60EE0A2DEF31E03F932F9324C02435310556
S1130A7009F070CEF70181818F3309F06BCEF2E07B
S1130A80EF0EF11CF98EE88EEA8DFB8DE080F1808B
S1130A906091A7027091A8028DE090E00E94EE0A96
S1130AA06091A7027091A8028AE090E00E94EE0A89
S1130AB0FF92EF92DF92CF920E942A0B0F900F9039
S1130AC00F900F9047CE8A3009F4FEC02F303105C5
S1130AD038F42F5F3F4F30934C0220934B028083B6
S1130AE06091A7027091A80290E00E94EE0AECC007
S1130AF08A89EB88FC88811116C080913F0290910D
S1130B004002E816F90609F4DFC0111107C0C70155
S1130B10880F991F880F991F0E949A02F092400231
S1130B20E0923F02D1C0823009F0CEC0F092480278
S1130B30E092470281E090E0F1E0EF16F2E0FF0678
S1130B4014F480E090E09093460280934502BCC088
S1130B508A89813041F118F08230A1F1B5C0113099
S1130B6019F424EF31E002C028EE33E0740181E08F
S1130B70E826892819F462E370E00BC02253310996
S1130B80A8EEB3E00E948C08A30192010E946A08B7
S1130B90B90180E00E942E07B70180E090E00E9436
S1130BA08206470191C0113009F08EC0809149023C
S1130BB090914A02892B09F485C085EA91E00E944C
S1130BC0400B80C062E370E082E00E942E078091B7
S1130BD045029091460220914302309144028217CB
S1130BE0930711F12091490230914A02232B61F0BD
S1130BF09F938F9385EB91E09F938F930E942A0B91
S1130C000F900F900F900F908091450290914602A3
S1130C10892B51F48FEF810F823030F481E090E022
S1130C200E944C0200E001C0012F80914502909186
S1130C304602909344028093430280E00E94E100C4
S1130C4082E00E94E1001017D9F18091490290914D
S1130C504A02892B01F1E02FF0E0EE0FFF1FE9506B
S1130C60FE4F81818F9380818F93E12FF0E0EE0F0F
S1130C70FF1FE950FE4F81818F9380818F9388EC11
S1130C8091E09F938F930E942A0B0F900F900F90E7
S1130C900F900F900F90023059F48FEF9FE00E9455
S1130CA09A0280E090E00E944C0261E070E004C08F
S1130CB0011106C060E070E082E090E00E948206CC
S1130CC0102F0DCD02E0C1CF012FFACF9F70FB0191
S1130CD09083818382E090E00895FB0120E42083E7
S1130CE024E0880F991F2A95E1F79183828383E09A
S1130CF090E008958CEF8AB996E094B98BB984E0BA
S1130D0085B90895FC01EE0FFF1F8E0F9F1FFC0194
S1130D10E05FFD4F808121E030E0018002C0220FBE
S1130D20331F0A94E2F7428150E0E82FF0E080A1FB
S1130D304617570711F0282B02C02095282320A31B
S1130D4008951F920F920FB60F921124DF92EF9223
S1130D50FF920F931F932F933F934F935F936F9340
S1130D607F938F939F93AF93BF93EF93FF93CF930F
S1130D70DF9300D000D0CDB7DEB780918F02909181
S1130D8090029093850080938400E12CF12C93E0F1
S1130D90D92E8701000F111F000F111F015B1D4F7A
S1130DA0F80180819181892BF1F082819381892BD3
S1130DB031F08281938101979383828314C01982D5
S1130DC01A821B821C82D982EA82BE016F5F7F4F26
S1130DD080914D0290914E020E946301892B19F07B
S1130DE0F80111821082FFEFEF1AFF0A80E1E81682
S1130DF0F10479F60F900F900F900F90DF91CF913F
S1130E00FF91EF91BF91AF919F918F917F916F91DE
S1130E105F914F913F912F911F910F91FF90EF9010
S1130E20DF900F900FBE0F901F90189590934E0275
S1130E3080934D027093900260938F0270938500AB
S1130E406093840010928000E1E8F0E08081877074
S1130E50482B408381E080936F0008950F931F9384
S1130E60CF93C82F8B010E94FC0084E0C89FF0013F
S1130E701124E15BFD4F1383028381E090E09183B1
S1130E808083CF911F910F910C9407011F920F92B1
S1130E900FB60F9211240F900FBE0F901F9018954C
S1130EA01F920F920FB60F9211240F900FBE0F9046
S1130EB01F9018951F920F920FB60F9211242F9323
S1130EC03F934F935F936F937F938F939F93AF93CE
S1130ED0BF93EF93FF93CF93DF9300D000D0CDB7B0
S1130EE0DEB78091C00087FF12C08091C6001982CE
S1130EF01A821B821C8291E099838A83BE016F5FF0
S1130F007F4F80919102909192020E9463010F9011
S1130F100F900F900F90DF91CF91FF91EF91BF91C0
S1130F20AF919F918F917F916F915F914F913F917D
S1130F302F910F900FBE0F901F9018954F925F92B4
S1130F406F927F928F929F92AF92BF92CF92DF92D5
S1130F50EF92FF92CF93DF9300D000D0CDB7DEB7EE
S1130F606A017B0190939202809391024A015B0192
S1130F7083E0880C991CAA1CBB1C8A95D1F760E0FD
S1130F8070E88CEF9AE0A50194010E946A08CA01F6
S1130F90B9016B5F7F4F8F4F9F4F2AE0422E512C38
S1130FA0612C712CA30192010E946A0829833A835F
S1130FB04B835C8334E0CC0CDD1CEE1CFF1C3A95A7
S1130FC0D1F760E070E88CEF9AE0A70196010E94E7
S1130FD06A08CA01B9016B5F7F4F8F4F9F4FA3010E
S1130FE092010E946A0829013A01A50194016981CC
S1130FF07A818B819C810E945A08705477FF03C0C8
S11310007195619571094B01770FAA08BB08A70177
S11310109601C301B2010E945A08705477FF03C0BD
S1131020719561957109CB01770FAA0BBB0B8816DB
S11310309906AA06BB0610F0920107C029813A81DD
S11310408091C00082608093C000215031092093B8
S1131050C4003093C50088E18093C1008091C10031
S113106080688093C1000F900F900F900F90DF91D4
S1131070CF91FF90EF90DF90CF90BF90AF909F9073
S11310808F907F906F905F904F9008959091C000E3
S113109095FFFCCF8093C6000895CF93C82F0E947C
S11310A04608CA3019F48DE00E94460880E090E0BA
S11310B0CF910895DB018F939F930E949B08BF916A
S11310C0AF91A29F800D911DA39F900DB29F900D93
S11310D011240895A1E21A2EAA1BBB1BFD010DC009
S11310E0AA1FBB1FEE1FFF1FA217B307E407F507D4
S11310F020F0A21BB30BE40BF50B661F771F881FB0
S1131100991F1A9469F760957095809590959B0145
S1131110AC01BD01CF010895A29FB001B39FC001EE
S1131120A39F700D811D1124911DB29F700D811D0F
S11311301124911D08950E948C08A59F900DB49FC1
S1131140900DA49F800D911D112408950F931F935A
S1131150CF93DF938230910510F482E090E0E09128
S1131160A302F091A40220E030E0A0E0B0E03097C8
S113117019F1408151810281138148175907C8F040
S11311808417950769F4109731F012960C9312970F
S113119013961C9327C00093A3021093A40222C0A9
S11311A02115310519F04217530718F49A01BD01AE
S11311B0EF01DF01F801DBCF21153105F9F0281B20
S11311C0390B2430310580F48A819B8161157105C6
S11311D021F0FB019383828304C09093A402809343
S11311E0A302FE01329644C0FE01E20FF31F819375
S11311F0919322503109398328833AC02091A10266
S11312003091A202232B41F4209102013091030179
S11312103093A2022093A102209100013091010198
S11312202115310541F42DB73EB740910401509189
S11312300501241B350BE091A102F091A202E217F3
S1131240F307A0F42E1B3F0B2817390778F0AC01E5
S11312504E5F5F4F2417350748F04E0F5F1F5093C2
S1131260A2024093A1028193919302C0E0E0F0E0D6
S1131270CF01DF91CF911F910F910895CF93DF9309
S1131280009709F481C0FC01329713821282A09165
S1131290A302B091A402109781F420813181820FBE
S11312A0931F2091A1023091A2022817390751F50A
S11312B0F093A202E093A10267C0ED0120E030E0C8
S11312C0CE17DF0740F44A815B819E014115510529
S11312D0F1F0EA01F5CFD383C28340815181840FB9
S11312E0951FC817D90759F488819981840F951FD0
S11312F00296918380838A819B81938382832115C3
S1131300310529F4F093A402E093A3023DC0E9015E
S1131310FB83EA8349915991C40FD51FEC17FD074C
S113132061F480819181840F951F0296E90199836C
S11313308883828193819B838A83E0E0F0E0129624
S11313408D919C911397009719F0FD01DC01F7CF63
S11313508D919C9111979D012E5F3F4F820F931F9A
S11313602091A1023091A2022817390769F430971D
S113137029F41092A4021092A30202C013821282D2
S1131380B093A202A093A102DF91CF910895A0E0AF
S1131390B0E0EDECF9E00C94C90D5C016B017A014D
S11313A06115710519F0FB0191838083E114F10447
S11313B029F0C7010297839708F0E5C0E50121965B
S11313C0F5011081812F90E00E94DD0A892B11F034
S11313D05E01F4CF1D3229F42196F501118101E05B
S11313E007C01B3221F4E5012296F501118100E0CA
S11313F0E114F10409F1F0E1EF16F10429F43FC01E
S113140010E3E114F10421F128E0E216F10401F102
S113141054F4E2E0EE16F10421F5812C912CA12C78
S1131420B0E4BB2E3EC0FAE0EF16F10439F020E13F
S1131430E216F104B1F430C0103319F1FAE0EF2EE2
S1131440F12CACEC8A2E982CA82CACE0BA2E29C036
S113145078E0E72EF12C812C912CA12CE0E1BE2E1A
S113146020C060E070E080E090E897010F2C000C51
S1131470440B550B0E946A0849015A0112C01033EB
S113148059F488818F7D883509F0BACF1981229665
S1131490026080E1E82EF12C812C912CA12C68E0D3
S11314A0B62E40E060E070E0CB0127010F2C000C69
S11314B066087708FE0150ED352E310E29E023151C
S11314C070F42FEB210F2A3118F439EC332E06C0B7
S11314D02FE9210F2A3118F529EA322E310E232D56
S11314E030E02E153F05DCF447FD16C0861697063E
S11314F0A806B90670F0A30192010E945A08630D70
S1131500711D811D911D61307105810520E89207CF
S113151010F04FEF01C041E021961081CBCF202F76
S11315202170C114D10471F0442329F02197F601EC
S1131530D183C08307C001FF19C02297F601D1836C
S1131540C08314C047FF12C0222329F060E070E07A
S113155080E090E804C06FEF7FEF8FEF9FE722E217
S113156030E03093AC022093AB0209C0222381F017
S113157090958095709561957F4F8F4F9F4F462F23
S1131580372F282F12C040E030E020E090E00DC05B
S113159097FFF5CF82E290E09093AC028093AB0288
S11315A06FEF7FEF8FEF9FE7EACF642F732F822FC8
S11315B0CDB7DEB7E1E10C94E50D91110C94510D1A
S11315C0803219F089508550C8F708959111089513
S11315D081568A5108F48052855808950F931F93B9
S11315E0CF93DF93FB01238121FD03C08FEF9FEF96
S11315F02CC022FF16C046815781248135814217B1
S1131600530744F4A081B1819D012F5F3F4F318383
S113161020838C93268137812F5F3F4F3783268326
S113162014C08B01EC01FB010084F185E02D0995C8
S1131630892BE1F6D80116968D919C911797019606
S113164017969C938E931697CE01DF91CF911F919D
S11316500F910895A0E0B0E0E0E3FBE00C94D80D16
S1131660AE014B5F5F4FFA0161917191AF018091BF
S1131670A7029091A8020E94700BE2E00C94F40D72
S11316800F931F93CF93DF93E091A702F091A802E9
S1131690238121FF1BC08C01D0E0C0E0F8018191BF
S11316A08F016091A7027091A802DB011896ED9159
S11316B0FC911997882331F00995892B79F3DFEF91
S11316C0CFEFECCF8AE00995892B19F08FEF9FEFCC
S11316D002C08D2F9C2FDF91CF911F910F91089500
S11316E0ABE0B0E0E6E7FBE00C94C80D6C017B01D5
S11316F08A01FC0117821682838181FFCCC1CE014D
S113170001963C01F6019381F70193FD859193FFC6
S113171081917F01882309F4BAC1853239F493FD9C
S1131720859193FF81917F01853229F4B60190E080
S11317300E94EE0AE7CF912C212C312CFFE1F31506
S1131740D8F08B3279F038F4803279F08332A1F416
S1131750232D20611DC08D3261F0803369F4232D67
S1131760216016C0832D8260382EE32DE4603E2E66
S11317702AC0F32DF8601DC037FC2DC020ED280FC2
S11317802A3040F08E32B9F436FC81C1232D206416
S1131790322E19C036FE06C08AE0989E200D112410
S11317A0922E11C0EAE02E9E200D1124222EF32D3C
S11317B0F0623F2E08C08C3621F4832D8068382EC9
S11317C002C0883641F4F70193FD859193FF81911E
S11317D07F018111B3CF982F9F7D9554933028F4C6
S11317E00C5F1F4F9FE399830DC0833631F083371D
S11317F071F0833509F059C021C0F80180818983D3
S11318000E5F1F4F88248394912C530113C0280129
S1131810F2E04F0E511CF801A080B18036FE03C0E7
S1131820692D70E002C06FEF7FEFC5010E945F0D6C
S11318304C018201F32DFF773F2E16C0280122E0D0
S1131840420E511CF801A080B18036FE03C0692D00
S113185070E002C06FEF7FEFC5010E94540D4C0190
S1131860F32DF0683F2E820133FC1BC0822D90E0E3
S113187088169906B0F4B60180E290E00E94EE0A60
S11318802A94F4CFF50137FC859137FE81915F01ED
S1131890B60190E00E94EE0A21102A9421E0821AF7
S11318A091088114910471F7E8C0843611F08936E7
S11318B041F5F80137FE07C060817181828193810F
S11318C00C5F1F4F08C060817181072E000C880BCC
S11318D0990B0E5F1F4FF32DFF763F2E97FF09C024
S11318E090958095709561957F4F8F4F9F4FF068CD
S11318F03F2E2AE030E0A3010E946A0D882E86184C
S113190045C0853731F4232D2F7EB22E2AE030E0F6
S113191025C0932D997FB92E8F36C1F018F48835E0
S113192079F0B5C0803719F0883721F0B0C0E92FBD
S1131930E061BE2EB4FE0DC0FB2DF460BF2E09C0C5
S113194034FE0AC0292F2660B22E06C028E030E0FB
S113195005C020E130E002C020E132E0F801B7FE2A
S113196007C060817181828193810C5F1F4F06C023
S11319706081718180E090E00E5F1F4FA3010E949F
S11319806A0D882E8618FB2DFF773F2E36FE0DC07C
S1131990232D2E7FA22E891458F434FE0BC032FC62
S11319A009C0832D8E7EA82E05C0B82CA32C03C09D
S11319B0B82C01C0B92CA4FE0FC0FE01E80DF11D26
S11319C08081803321F49A2D997EA92E09C0A2FE2C
S11319D006C0B394B39404C08A2D867809F0B394F6
S11319E0A3FC11C0A0FE06C0B21488F4280C922CEB
S11319F09B180EC0B21460F4B60180E290E00E941D
S1131A00EE0AB394F7CFB21418F42B1802C0982C32
S1131A10212CA4FE10C0B60180E390E00E94EE0ADF
S1131A20A2FE17C0A1FC03C088E790E002C088E5CD
S1131A3090E0B6010CC08A2D867859F0A1FE02C050
S1131A408BE201C080E2A7FC8DE2B60190E00E9427
S1131A50EE0A891438F4B60180E390E00E94EE0A9D
S1131A609A94F7CF8A94F301E80DF11D8081B601B1
S1131A7090E00E94EE0A8110F5CF222009F442CEB4
S1131A80B60180E290E00E94EE0A2A94F6CFF601B5
S1131A908681978102C08FEF9FEF2B96E2E10C9431
S1131AA0E40D992788270895FC0105906150704042
S1131AB00110D8F7809590958E0F9F1F0895FC0113
S1131AC06150704001900110D8F7809590958E0F69
S1131AD09F1F0895FA01AA27283051F1203181F17E
S1131AE0E8946F936E7F6E5F7F4F8F4F9F4FAF4F22
S1131AF0B1E03ED0B4E03CD0670F781F891F9A1F35
S1131B00A11D680F791F8A1F911DA11D6A0F711DE8
S1131B10811D911DA11D20D009F468943F912AE0F4
S1131B20269F11243019305D3193DEF6CF010895DC
S1131B30462F4770405D4193B3E00FD0C9F7F6CF0D
S1131B40462F4F70405D4A3318F0495D31FD4052D5
S1131B50419302D0A9F7EACFB4E0A695979587956B
S1131B6077956795BA95C9F700976105710508954A
S1131B709B01AC010A2E06945795479537952795F6
S1131B80BA95C9F7620F731F841F951FA01D08958E
S1131B902F923F924F925F926F927F928F929F9279
S1131BA0AF92BF92CF92DF92EF92FF920F931F9367
S1131BB0CF93DF93CDB7DEB7CA1BDB0B0FB6F89418
S1131BC0DEBF0FBECDBF09942A88398848885F8458
S1131BD06E847D848C849B84AA84B984C884DF80C9
S1131BE0EE80FD800C811B81AA81B981CE0FD11DAD
S1131BF00FB6F894DEBF0FBECDBFED010895F89483
S1051C00FFCF10
S1131C020000AD02200000000002000000004D08A8
S1131C120000000068016C01436F6E764669666FCE
S1131C22004572726F72204932435F5354415254D9
S1131C32004572726F72204932435F534C415F41D7
S1131C42434B004572726F72204932435F444154E0
S1131C52415F41434B005365742073776974636831
S1131C6220746F2025730A004F4646004F4E0053DE
S1131C72657420506F77657220746F202575206417
S1131C8269676974730A0025732025730A004F4B30
S1131C923A25303475004F4B3A2575004F4B004FAF
S1131CA24B3A25730052656D6F74652074696D65D6
S1131CB26F757421005077725377697463685F6932
S1131CC26E203D2025640A005374617465206368A4
S1131CD2616E67652022257322203D3E20222573F2
S1131CE2220A004E6F726D616C0052656D6F7465ED
S1131CF2004572726F7200E301EA01F10176312E3E
S1131D02310048656E64692D436F6E74726F6C00A6
S1131D120502010B06010B07010B02010B03010B68
S10B1D2204010B050105010198
S9030000FC
